:020000040800F2
:1000000000040020E1010008450E0008490E000828
:100010009D0E0008490E0008710E0008E30100085B
:10002000E3010008E3010008E3010008812F000854
:10003000E3010008E3010008E3010008E301000810
:10004000E3010008E3010008E3010008E301000800
:10005000E3010008E3010008E5310008113200085F
:100060003D3200086932000895320008E3010008BB
:10007000E3010008E3010008E3010008E3010008D0
:10008000E3010008E3010008E3010008E3010008C0
:10009000E3010008E3010008E3010008C1320008A1
:1000A000E3010008E3010008E3010008E3010008A0
:1000B000E3010008E3010008E3010008E301000890
:1000C000E3010008E3010008E3010008E301000880
:1000D000E3010008E3010008E3010008E301000870
:1000E00029330008E3010008E3010008E3010008E8
:1000F000E3010008E3010008E3010008E301000850
:10010000E3010008E3010008FD2F0008E3010008F7
:10011000E3010008E3010008E3010008E30100082F
:10012000E3010008E3010008E3010008E30100081F
:10013000E3010008E3010008E3010008E30100080F
:10014000E3010008E3010008E3010008C9260008F4
:10015000E3010008E3010008E3010008E3010008EF
:10016000E3010008E3010008E3010008E3010008DF
:10017000E3010008E3010008E3010008E3010008CF
:10018000E3010008E3010008E3010008E3010008BF
:10019000E3010008E3010008E3010008E3010008AF
:1001A000E3010008E3010008E3010008E30100089F
:1001B000E3010008E3010008E3010008E30100088F
:1001C000E3010008E3010008E3010008E30100087F
:1001D000E3010008E3010008E3010008E30100086F
:1001E00002E000F000F8FEE772B6394880F30888B4
:1001F000384880F3098838484EF60851CEF200019D
:10020000086040F20000CCF200004EF63471CEF2ED
:1002100000010860BFF34F8FBFF36F8F40F2000003
:10022000C0F2F0004EF68851CEF200010860BFF334
:100230004F8FBFF36F8F4FF00000E1EE100A4EF6C4
:100240003C71CEF200010860062080F31488BFF3F1
:100250006F8F01F001FF02F029FE4FF055301F496A
:100260001B4A91423CBF41F8040BFAE71C49194A6A
:1002700091423CBF41F8040BFAE71A491A4A1B4B5A
:100280009A423EBF51F8040B42F8040BF8E70020F5
:100290001749184A91423CBF41F8040BFAE701F0B4
:1002A000DFFE02F05FFE144C144DAC4203DA54F84A
:1002B000041B8847F9E700F03FF8114C114DAC42A0
:1002C00003DA54F8041B8847F9E701F0C7BE0000C1
:1002D000000400200024002000000008000000208E
:1002E00000040020483700080024002028240020B3
:1002F0002824002018300020E0010008E001000858
:10030000E0010008E00100082DE9F04F2DED108A12
:10031000C1F80CD0C3689D46BDEC108ABDE8F08FD3
:10032000002383F311882846A047002001F018FB22
:1003300001F0C8FA00DFFEE71C4B6FF07F0270B5DA
:100340001A7004225A706FF03F0200245A720F2272
:100350009C70DC701C715C719C71DC711C729A72F7
:10036000DC7201F04BFE064601F070FE054650B906
:100370000F4B9E4217D001339E4241F2883412BF88
:10038000054600240125002001F042FE0DB100F0D9
:10039000B5F800F02BFD00F0F5FB204600F00CF95D
:1003A00000F0ACF8F9E70446EDE700BF2824002090
:1003B000010007B008B500F087FBA0F12003584208
:1003C000584108BD07B5054B02211B88ADF8043024
:1003D00001A800F0C7FB03B05DF804FB0C34000873
:1003E000064991F8243033B100230822086A81F8C5
:1003F000243000F0E9BB0120704700BF48240020F2
:100400002DE9F84F234C94F82430054688461746CA
:100410008BBB2E46DFF87C90002F38D094F824A0B8
:10042000BAF1000F05D12022FF214846266200F0D4
:10043000CBFCCAF10805BD4228BF3D465FFA85FBEB
:10044000AD0041462A4604EB8A0000F093FC94F884
:100450002430A7EB0B079B445FFA8BFBBBF1080F23
:100460002E44A844FFB284F824B0D5D1FFF7B8FFDA
:100470000028D1D108E0266A06EB8306B042C9D035
:10048000FFF7AEFF0028C4D10020BDE8F88F01209F
:10049000BDE8F88F4824002010B5202383F311888D
:1004A0001248C3680BB101F0E1FA0023104A0F486B
:1004B0004FF47A7101F09EFA002383F311880D4CFA
:1004C000236813B12368013B2360636813B1636839
:1004D000013B6360084B1B7833B9636823B9022082
:1004E00000F034FC3223636010BD00BF34240020D0
:1004F00099040008782500207024002010B5254BB1
:10050000254953F8042F013200D110BD8B42F8D198
:10051000224C234B22689A423AD9224B9B6803F122
:10052000006303F580439A4232D2002000F044FB7E
:100530001D4B0220187000F0F9FB1C4B1A6C0022B6
:100540001A64196E1A66196E596C5A64596E5A6695
:100550005A6E5A6942F080025A615A6922F080024A
:100560005A615A691A6942F000521A611A6922F0F6
:1005700000521A611B6972B60D4A0E4B13601B685C
:100580002268202181F311889D4683F30888104753
:1005900010BD00BFFC3F00081C40000804400008DC
:1005A000FF3F00082824002070240020003802406B
:1005B00008ED00E0004000082DE9F04F99B0B34C81
:1005C00001902022FF2110A8A66800F0FDFBB04A90
:1005D0001378A346A3B9AF480121C360117020234B
:1005E00083F31188C3680BB101F040FA0023AA4AD3
:1005F000A8484FF47A7101F0FDF9002383F31188C4
:10060000019B13B1A54B019A1A60A54AA349019F0A
:100610000292002313704B6099461C461D46984673
:10062000012000F083FB002F00F012829B4B1B681F
:10063000002B40F00D8219B0BDE8F08F0220FFF7CB
:10064000B9FE002840F0FB81019BB9F1000F08BF03
:100650001F46944B1B88ADF82C3002210BA800F0EC
:1006600081FADDE74FF47A7000F02EFA031E03934F
:10067000EADB0220FFF79EFE82460028E4D0039BBF
:10068000581E042800F2DD81DFE800F0030E11148B
:10069000170018A8052340F8343D042100F062FA41
:1006A00054464FF0000856E004217848F6E704214C
:1006B0007D48F3E704217D48F0E71C24204600F044
:1006C0007DFA04340B9004210BA800F04BFA2C2C7B
:1006D000F4D1E5E7002DB7D0002CB5D00220FFF70C
:1006E00069FE0546002800F0AF8101206C4C00F047
:1006F00063FA0220207000F019FB4FF000095FFA46
:1007000089FA504600F068FA074658B1504600F0A2
:1007100073FA09F101090028F1D12C46A9460027F6
:10072000634B97E701230220237000F0EDFA3E4669
:10073000DBF808309E4206D2304600F03FFA013026
:10074000EBD10436F4E7029B00261E70534BA946FA
:100750005E602C46374600F03FFB15B1002C18BFF9
:100760000027FFF72FFE5BE7002D3FF46DAF002C55
:100770003FF46AAF029B0220187000F0D7FA3220D3
:1007800000F0A2F9B0F1000AC0F25E811AF0030590
:1007900040F05A81DBF8082006EB0A03934200F28E
:1007A0005381BAF5807F00F24F8155450DDA4FF441
:1007B0007A7000F089F90490049B002BC0F2448108
:1007C0003C4A049BAB540135EFE7C820FFF7F2FD2C
:1007D0000546002800F038811F2E11D8C6F12004EC
:1007E000544528BF544610AB26F003002246314939
:1007F000184400F0BFFA2246FF212E4800F0E4FA28
:100800004FEAAA0A5FFA8AF22A493046FFF7F8FD52
:100810000446002800F01A8106EB8A0605469AE78E
:100820000220FFF7C7FD00283FF40EAFFFF7D8FD09
:1008300000283FF409AF4FF0000A5346DBF80820C8
:1008400092451CD2BAF11F0F12D8109A01320FD064
:100850002AF0030218A90A4452F8202C0B921846D9
:1008600004220BA900F02EFB0AF1040A0346E5E777
:100870005046039300F0A2F9039B0B90EFE718A8F2
:10088000042140F84C3D00F06DF964E72824002075
:1008900074250020342400209904000878250020C5
:1008A000702400200E3400082C2400203024002066
:1008B000103400087424002018A8002340F8343DA8
:1008C000642100F02BF900287FF4BEAE0220FFF770
:1008D00071FD00283FF4B8AE0B9800F09FF918ABFB
:1008E00043F8480D04211846CDE718A8002340F826
:1008F000343D642100F012F900287FF4A5AE0220F7
:10090000FFF758FD00283FF49FAE0B9800F094F9D4
:1009100018AB43F8440DE5E70220FFF74BFD002834
:100920003FF492AE00F08EF918AB43F8400DD9E7D2
:100930000220FFF73FFD00283FF486AE0BA91420EC
:1009400000F086F9824618A8042140F83CAD00F07A
:1009500009F951460BA896E7322000F0B5F8B0F13E
:10096000000AFFF671AE1AF0030F7FF46DAEDBF8EC
:1009700008200AEB080393423FF666AE0220FFF719
:1009800019FD00283FF460AE2AF0030AC244D045A6
:100990003FF4E1AE404600F011F904210A900AA8A4
:1009A00000F0E0F808F10408F1E74FF47A70FFF77F
:1009B00001FD00283FF448AEFFF712FD00283FF488
:1009C000AFAE109B01330CD0082210A90020FFF716
:1009D00017FD00283FF4A4AE2022FF2110A800F04C
:1009E000F3F9FFF7EFFC374800F0C0FF23E6002DD6
:1009F0003FF42AAE002C3FF427AE18A8002340F89D
:100A0000343D642100F08AF8824600287FF41CAE51
:100A10000220FFF7CFFC00283FF416AE0390FFF74B
:100A2000D1FC41F2883000F0A1FF0B9800F008FAE9
:100A300000F0D2F9039B57461C461D46F0E50546DB
:100A400089E64FF00008FFE52546FDE52C4667E600
:100A5000002000F039F80490049B002BFFF6E3AD72
:100A6000012000F051F9049B213B122B3FF6D8AD39
:100A700001A252F823F000BF3D06000865060008F9
:100A8000D5060008210600082106000821060008F6
:100A9000690700085909000821080008B90800087A
:100AA000EB080008190900082106000831090008B0
:100AB00021060008AB0900085707000821060008B6
:100AC000EF090008A086010037B5114B1A780132F2
:100AD000D2B20024012A01468DF8074011D80D48F2
:100AE00003681D6A4FF47A734B4301220DF107012D
:100AF000A847012805D1084B9DF807001C7003B0DA
:100B000030BD4FF4FA7000F031FF4FF0FF30F6E7E0
:100B100000240020482600208425002038B50E4BF4
:100B20001A780132D2B2012A05460ED80B48036862
:100B30001C6A4FF47A734B4304222946A0470428C9
:100B400003D1074B0020187038BD4FF4FA7000F045
:100B50000DFF4FF0FF3038BD002400204826002054
:100B60008425002030B4054C2368DD69044B0A4617
:100B7000AC460146204630BC604700BF48260020F6
:100B8000A086010070B501F03DF9094C094E2070B6
:100B9000002530682378834208D901F02DF93368A5
:100BA00005440133B5F5804F3360F2D370BD00BF0B
:100BB000852500208025002001F0D2B900F10060D9
:100BC00000F580400068704700F10060920000F579
:100BD000804001F05DB90000054B1A68054B1B7899
:100BE0009B1A834202D9104401F006B900207047D5
:100BF000802500208525002038B5074D044628684B
:100C0000204401F001F928B928682044BDE83840A3
:100C100001F012B938BD00BF8025002010F0030399
:100C200008D1B0F5007F05D800F10050A0F50840CC
:100C30000068704700207047014BC058704700BFE4
:100C4000107AFF1F014B1868704700BF002004E0B6
:100C500070B52A4B1C68C4F30B03240C63B140F23B
:100C60001342934231D040F2194293422FD040F2C6
:100C7000214293422DD10323214A0C2505FB032356
:100C80005D6893F9082042F201039C4224D0B4F538
:100C9000805F23D041F201039C4221D041F2030343
:100CA0009C421FD041F207039C4208BF3122441EE0
:100CB0000C44013D0B46A3421ED215F9016F581C8E
:100CC00096B1034600F8016CF5E70123D4E702234F
:100CD000D2E73F220B4DD6E73322E3E74122E1E79B
:100CE0005A22E4E75922E2E72C2584421D7001D9FB
:100CF000981C5A70401A70BD1846FBE7002004E0AB
:100D00002034000814340008022804D1054B4FF0A9
:100D100080429A6170470128FCD14FF40012024BC7
:100D2000F7E700BF000C024000080240022804D18F
:100D3000044B4FF480429A6170470128FCD1202275
:100D4000014BF8E7000C024000080240022805D1E0
:100D5000064A536983F48043536170470128FCD1EC
:100D6000034A536983F02003F6E700BF000C0240FA
:100D70000008024010B50023934203D0CC5CC45459
:100D80000133F9E710BD000030B5441E14F9010F1E
:100D90000B4660B193F90050854201F1010106D183
:100DA0001AB993F90020801A30BD013AEEE7002A03
:100DB000F7D1104630BD000002460346981A13F9D9
:100DC000011B0029FAD1704702440346934202D026
:100DD00003F8011BFAE77047024B1A78024B1A70AE
:100DE000704700BF842500200024002038B5104D36
:100DF000104C284600F002F92146284600F02AF956
:100E000024680D48626DD2F8043843F00203C2F83A
:100E1000043800F0ABFD0949204600F027FA626D66
:100E2000D2F8043823F00203C2F8043838BD00BFFA
:100E300048260020EC34000840420F001C35000812
:100E400070470000FEE7000000B59BB0EFF309819A
:100E500068226846FFF78EFFEFF30583034B9A6B1A
:100E60009A6A9A6A9A6A9A6A9B6AFEE700ED00E0BB
:100E700000B59BB0EFF3098168226846FFF77AFF5F
:100E8000EFF30583044B9A6B9A6A9A6A9A6A9A6A94
:100E90009A6A9B6AFEE700BF00ED00E000B59BB0D8
:100EA000EFF3098168226846FFF764FFEFF30583DB
:100EB000034B5A6B9A6A9A6A9A6A9A6A9B6AFEE725
:100EC00000ED00E030B5084D0A4491420BD011F816
:100ED000013B09245840013CF7D040F300032B406C
:100EE00083EA5000F7E730BD2083B8ED00230449C2
:100EF0001A465A50C8180833802B4260F9D17047FF
:100F000088250020026843681143016003B1184737
:100F10007047000013B5446BD4F894341A68117804
:100F2000042915D1217C022912D1197912890123B2
:100F30008B4013420CD101A904F14C0001F02AFEB0
:100F4000D4F89444019B21790246206800F0DAF934
:100F500002B010BD143001F0ADBD00004FF0FF3302
:100F6000143001F0A7BD00004C3001F07FBE00003E
:100F70004FF0FF334C3001F079BE0000143001F027
:100F80007BBD00004FF0FF31143001F075BD000053
:100F90004C3001F04BBE00004FF0FF324C3001F0FE
:100FA00045BE0000D0F8942438B513681978042998
:100FB000054601D0012038BD017C0229FAD1127901
:100FC0005C89012090400440F4D105F1140001F047
:100FD0000DFD02460028EDD0D5F894544FF48073EF
:100FE0002868697900F07CF9204638BD406BFFF72E
:100FF000D9BF000000207047704700007FB5124B3A
:101000000360002343608360C360012502260F4B09
:10101000057404460290019300F18402294600966B
:101020004FF48073143001F0BDFC094B019302941E
:1010300000964FF4807304F52372294604F14C00A6
:1010400001F084FD04B070BD70340008ED0F00089D
:10105000150F00080B68202282F311880A7903EB30
:10106000820290614A79093243F822008A7912B1EA
:1010700003EB8203986102230374C0F894140023E5
:1010800083F311887047000038B5037F044613B11D
:1010900090F85430ABB9201D01250221FFF732FF33
:1010A00004F1140025776FF0010100F087FC84F84B
:1010B000545004F14C006FF00101BDE8384000F0DD
:1010C0007DBC38BD10B5012104460430FFF71AFF7E
:1010D0000023237784F8543010BD000038B504464F
:1010E0000025143001F076FC04F14C00257701F066
:1010F00045FD201D84F854500121FFF703FF2046D1
:10110000BDE83840FFF74EBF90F8443003F060036D
:10111000202B19D190F84520212A0AD0222A4FF0FD
:1011200000030ED0202A0FD1084A82630722C2632F
:1011300004E0064B83630723C36300230364012099
:1011400070478363C363F9E70020704701240020E0
:10115000D0F8943437B51A681178042904461AD1A6
:10116000017C022917D11979128901238B4013427E
:1011700011D100F14C05284601F0C0FD58B101A97C
:10118000284601F007FDD4F89444019B21790246DA
:10119000206800F0B7F803B030BD000000EB810319
:1011A000F7B59C6905460E46F4B1202383F31188F8
:1011B00005EB8607201D0821FFF7A4FEFB685B698D
:1011C0001B684C3413B1204601F0F2FC01A9204603
:1011D00001F0E0FC024648B1019B3146284600F090
:1011E00091F8002383F3118803B0F0BDFB685A69BE
:1011F0001268002AF5D01B8A013B1340F1D105F19A
:101200004402EAE7093138B550F82140DCB1202327
:1012100083F31188D4F894241368527903EB820382
:10122000DB689B695D6845B104216018FFF76AFEC1
:10123000294604F1140001F0E3FB2046FFF7B2FE5B
:10124000002383F3118838BD7047000000F08EBF83
:101250000123037000234360C36183620362C3629E
:1012600043620363038143817047000038B504463D
:10127000202383F3118800254160C5600561456125
:10128000856100F083FF0223237085F3118838BD48
:1012900070B500EB810305465069DA600E461446CE
:1012A00018B110220021FFF78FFDA06918B110229C
:1012B0000021FFF789FD31462846BDE8704001F066
:1012C0002FB80000028902F001020281428902F077
:1012D00001024281002202614261826101F0B4B8E0
:1012E000F0B400EB81044789E4680125A4698D40CE
:1012F0003D43458123600023A2606360F0BC01F0A0
:10130000CFB80000F0B400EB81040789E468012540
:1013100064698D403D43058123600023A2606360C2
:10132000F0BC01F049B9000070B502230025044665
:101330000370A0F84C5080F84E5080F84F50058153
:101340004581C56005614561856180F8345000F0D4
:1013500083FF63681B6823B129462046BDE87040BF
:10136000184770BD436802781B6880F8502005223A
:1013700002700BB10421184770470000436890F8D1
:1013800050201B6802700BB1052118477047000000
:1013900090F8343070B5044613B1002380F834302F
:1013A00004F14402204601F071F863689B6863BB56
:1013B00094F8445015F0600615D194F8453005F0C6
:1013C0007F0545EA032540F202339D4200F00E817D
:1013D0005BD8022D00F0DC803FD8002D00F0878024
:1013E000012D00F0CF800021204601F0A7FA002156
:1013F000204601F099FA63681B6813B10621204664
:101400009847062384F8343070BD2046984700285A
:10141000CED094F84B2094F84A3043EA0223E26B92
:10142000934238BFE36394F94430E56B002B4FF0EF
:10143000200380F2FD80002D00F0EC80092284F86A
:10144000342083F311880021E36BA26B2046FFF761
:1014500059FF002383F3118870BDB5F5817F00F03B
:10146000B180B5F5407F49D0B5F5807FBBD194F808
:101470004630012BB7D1B4F84C3023F00203A4F866
:101480004C30A663E6632664C3E740F201639D42E5
:101490001ED8B5F5C06F3BD2B5F5A06FA3D1B4F897
:1014A0004430B3F5A06F0ED194F8463084F84E3036
:1014B000204600F029FF63681B6813B10121204614
:1014C0009847032323700023A363E3632364A0E707
:1014D000B5F5106F32D040F602439D4252D0B5F5BB
:1014E000006F80D104F14F03A363012324E004F1D2
:1014F0004C03A3630223E36325648AE794F8463030
:10150000012B7FF470AFB4F84C3043F00203B6E720
:1015100094F84920616894F848304D6894F8471071
:1015200043EA0223204694F84620A84700283FF4C7
:101530005AAF4368A3630368E363A4E72378042BEB
:1015400010D1202383F311882046FFF7BBFE86F3DA
:101550001188636884F84F601B68032121700BB108
:101560002046984794F84630002BACD084F84F3092
:101570000423237063681B68002BA4D0022120463B
:101580009847A0E7374BA3630223E36300239DE75B
:1015900094F8481011F0800F204601F00F010ED092
:1015A00000F066FF012806D002287FF41CAF2E4B06
:1015B000A363E06367E72D4BA363E56363E700F094
:1015C00049FFEFE794F84630002B7FF40CAF94F816
:1015D000483013F00F013FF476AF1A06204602D5CB
:1015E00001F0C0F96FE701F0B3F96CE794F8463009
:1015F000002B7FF4F8AE94F8483013F00F013FF45D
:1016000062AF1B06204602D501F098F95BE701F0B6
:101610008BF958E7142284F8342083F311882B4681
:101620002A4629462046FFF75BFE85F3118870BDE8
:101630005DB1152284F8342083F311880021E36B17
:10164000A26B2046FFF74CFE03E70B2284F8342000
:1016500083F311882B462A4629462046FFF752FE7F
:10166000E3E700BFA0340008983400089C34000869
:1016700038B590F834300446152B29D8DFE803F04C
:101680003E28282828283E28280B293928282828B9
:10169000282828283E3E90F84B1090F84A20C36B2B
:1016A00042EA01229A4214D9C268128AB3FBF2F5C7
:1016B00002FB15356DB9202383F311882B462A468A
:1016C0002946FFF71FFE85F311880A2384F834307A
:1016D00038BD142384F83430202383F31188002389
:1016E0001A4619462046FFF7FBFD002383F31188B5
:1016F00038BD036C03B198470023E7E7002101F0F0
:101700001DF90021204601F00FF963681B6813B131
:101710000621204698470623D8E7000090F8342099
:10172000152A38B5044622D80123934040F6416279
:1017300013421DD113F480150FD19B0217D50B2333
:1017400080F83430202383F311882B462A4629461B
:10175000FFF7D8FD85F3118838BDC3689B695B68C6
:101760002BB9036C03B19847002384F8343038BD9B
:10177000002101F0E3F80021204601F0D5F863686C
:101780001B6813B10621204698470623EDE70000A9
:10179000024B00221B605B609A60704708260020A5
:1017A000002303748268054B1B6899689142FBD241
:1017B0005A68036042601060586070470826002035
:1017C00008B5202383F31188037C032B05D0042B59
:1017D0000DD02BB983F3118808BD436900221A602C
:1017E0004FF0FF334361FFF7DBFF0023F2E790E8A0
:1017F0000C001A6002685360F2E7000000230374D3
:101800008268054B1B6899689142FBD85A6803604F
:10181000426010605860704708260020054B196927
:101820000874186802681A60536018610123037411
:10183000FEF76ABD0826002030B54B1C87B0054670
:101840000A4C10D023690A4A01A800F0D3F82846B0
:10185000FFF7E4FF049B13B101A800F007F9236927
:10186000586907B030BDFFF7D9FFF8E70826002018
:10187000C117000838B50C4D41612B6981689A6821
:101880009142044603D8BDE83840FFF789BF1846A7
:10189000FFF786FF01232C61014623742046BDE833
:1018A0003840FEF731BD00BF08260020044B1A68FF
:1018B0001B6990689B68984294BF00200120704784
:1018C0000826002010B5084C236820691A68226099
:1018D0005460012223611A74FFF790FF01462069CA
:1018E000BDE81040FEF710BD0826002082600222ED
:1018F00002740022427470478368A3F17C0243F8AB
:101900000C2C026943F83C2C426943F8382C074AF6
:1019100043F81C2CC26843F8102C022203F8082C50
:10192000002203F8072CA3F11800704721030008D8
:1019300010B5202383F31188FFF7DEFF0021044652
:10194000FFF798FF002383F31188204610BD0000A5
:10195000024B1B6958610F20FFF760BF082600206B
:10196000202383F31188FFF7F3BF000008B5014679
:10197000202383F311880820FFF75EFF002383F301
:10198000118808BD49B1064B42681B6918605A604E
:10199000136043600420FFF74FBF4FF0FF307047E4
:1019A000082600200368984206D01A68026050603A
:1019B00059611846FFF7F4BE7047000038B5044679
:1019C0000D462068844200D138BD036823605C6006
:1019D0004561FFF7E5FEF4E7054B03F114025A6198
:1019E0009A614FF0FF32DA6100221A62704700BF3D
:1019F00008260020F8B503611A4BC2605C6A1A4BD6
:101A00001A46022952F8145F38BF02219542064651
:101A10001F460AD1586198611C620560456081606B
:101A20000819BDE8F84001F08BB9186AAB68241AB0
:101A30000C1902D3E41A2D6804E09C4202D220441F
:101A400001F08EF9AB689C42F4D86B687360356026
:101A50001E606E60B460A9684FF0FF33091BA96077
:101A6000FB61F8BD000C00400826002010B41A4CA1
:101A7000234653F8141F814210D0416802680A605F
:101A8000026851609A424FF00001C16003D0936830
:101A900081680B4493605DF8044B70470A6862618B
:101AA00000209A425360C86003D15DF8044B01F0F6
:101AB00051B99368886803449360084A206A526A5F
:101AC000121A9342E7D9991A012998BF931C184416
:101AD0005DF8044B01F044B908260020000C0040DA
:101AE00000207047FEE70000704700004FF0FF3015
:101AF00070470000022906D0032906D001290648B4
:101B000018BF0020704705487047032A9ABF044851
:101B100000EBC20000207047783500082C35000823
:101B20000824002070B59AB001AD06460846294643
:101B3000144600F095F82846FFF73EF9C0B2431C62
:101B40005B0086E8180023700323637000230234CF
:101B50001946DAB2904204F1020401D81AB070BDFD
:101B6000EA5C04F8022C04F8011C0133F1E70000E0
:101B700008B5202383F311880348FFF7E9FA00230F
:101B800083F3118808BD00BF4826002010B5044625
:101B9000052916D8DFE801F016150316161D2023B7
:101BA00083F311880E4A0121FFF772FB20460D4A8C
:101BB0000221FFF76DFB0C48FFF790FA002383F337
:101BC000118810BD202383F311880748FFF75CFAC2
:101BD000F4E7202383F311880348FFF773FAEDE756
:101BE000A4340008C83400084826002038B50C4D3D
:101BF0000C4C0D492A4604F10800FFF793FF05F14C
:101C0000CA0204F110000949FFF78CFF05F5CA72FA
:101C100004F118000649BDE83840FFF783BF00BF54
:101C2000102B002008240020F4340008053500089B
:101C30001035000870B5044608460D46FFF7BCF89D
:101C4000C6B22046013403780BB9184670BD32463F
:101C50002946FFF799F80028F3D1012070BD000054
:101C60002DE9F84F05460C46FFF7A6F82C49C6B2F9
:101C70002846FFF7DFFF08B10436F6B229492846A7
:101C8000FFF7D8FF08B11036F6B2632E0DD8DFF893
:101C90009090DFF890A0DFF89880DFF898B0224F9E
:101CA0002E7846B92670BDE8F88F29462046BDE853
:101CB000F84F01F0A3BB252E2DD107224946284617
:101CC000FFF762F850B93B6823607B6863603B892B
:101CD0002381BB7AA37207350B34E1E70822514612
:101CE0002846FFF751F8B0B9104BA21C13F8011F9A
:101CF00009095B4511F8081002F8021C197801F077
:101D00000F0102F1020211F8081002F8031CEDD1D4
:101D100018340835C4E7267001350134C0E700BF28
:101D20009835000810350008A03500080F7AFF1F0D
:101D3000AC3500081B7AFF1FBFF34F8F024AD368F0
:101D4000DB03FCD4704700BF003C024008B5094BE0
:101D50001B7873B9FFF7F0FF074B1A69002ABFBF62
:101D6000064A5A6002F188325A601A6822F4806288
:101D70001A6008BD6E2D0020003C0240230167451B
:101D800008B50B4B1B7893B9FFF7D6FF094B1A69BF
:101D900042F000421A611A6842F480521A601A68CE
:101DA00022F480521A601A6842F480621A6008BDF8
:101DB0006E2D0020003C02400B2870B513D80B4A52
:101DC0000B4C137863B90B4E4FF0006144F82310AD
:101DD00056F8235001330C2B2944F7D101231370FB
:101DE00054F8200070BD002070BD00BFA02D002061
:101DF000702D0020C0350008014B53F820007047BB
:101E0000C03500080C2070470B2810B5044601D9D6
:101E1000002010BDFFF7D0FF064B53F824301844C4
:101E2000C21A0BB9012010BD12680132F0D1043B77
:101E3000F6E700BFC03500080B2810B5044621D8CE
:101E4000FFF77AFFFFF782FF0F4AF323D360C30047
:101E5000DBB243F4007343F002031361136943F4EC
:101E600080331361FFF768FFFFF7A6FF074B53F8B6
:101E7000241000F0DDF8FFF783FF2046BDE8104096
:101E8000FFF7C2BF002010BD003C0240C035000873
:101E90002DE9F84312F00103154640D18218B2F142
:101EA000016F3CD22C4B1B6813F0010337D02B4C35
:101EB000FFF74CFFF323E360FFF73EFF40F20127FB
:101EC000032D01D9830713D0244C0F46401A40F24A
:101ED0000118EB1B0B44012B00EB0706236924D8E8
:101EE00023F001032361FFF74BFF0120BDE8F883D6
:101EF000236923F44073236123693B43236151F831
:101F0000046B0660BFF34F8FFFF716FF03689E4216
:101F100008D0236923F001032361FFF731FF00207C
:101F2000BDE8F883043D0430CAE723F4407323611D
:101F3000236943EA08032361B94637F8023B33803B
:101F4000BFF34F8FFFF7F8FE3688B9F80030B6B20E
:101F5000B342BED0DDE700BF00380240003C024083
:101F6000084908B50B7828B153B9FFF7EFFE0123F4
:101F70000B7008BD23B1BDE808400870FFF700BF33
:101F800008BD00BF6E2D002010B50244064B043979
:101F9000D2B2904200D110BD441C00B253F82000D0
:101FA00041F8040FE0B2F4E750280040104B30B580
:101FB0001C6F240407D41C6F44F400741C671C6F4E
:101FC00044F400441C670B4C236843F48073236083
:101FD0000244094B0439D2B2904200D130BD441CB6
:101FE00000B251F8045F43F82050E0B2F4E700BFBC
:101FF00000380240007000405028004007B5012220
:1020000001A90020FFF7C0FF019803B05DF804FBB1
:1020100013B50446FFF7F2FFA04206D002A9012241
:1020200041F8044D0020FFF7C1FF02B010BD0000D1
:1020300070470000034B1B689B0042BF024B01220C
:102040001A70704774380240A12D0020014B187897
:10205000704700BFA12D002070470000FEE7000080
:10206000084A094B09498B4204D3094A002193428B
:1020700005D3704752F8040F43F8040BF3E743F815
:10208000041BF4E76C3700081830002018300020DB
:1020900018300020836D30B500229D68446D1146D4
:1020A0004FF0FF3004EB421301329542C3F80019A0
:1020B000C3F81019C3F80809C3F8001BC3F8101BB4
:1020C000C3F8080BEED24FF00113C4F81C3830BD32
:1020D000890141F02001016103699B06FCD41220B3
:1020E00000F0CABE204B03EB80022DE9F047D2F886
:1020F0000CE05D6DDEF81420461CD2F800C005EB44
:10210000063605EB4018516861450BD3D5F83428E5
:10211000012303FA00F022EA0000C5F8340818464B
:10212000BDE8F087BEF81040ACEB0103A34228BF26
:102130002346D8F81849A4B2B3EB840F10D894689A
:102140001F46A4F1040959F804AFC6F800A0042FF3
:1021500001D9043FF7E71C440B4494605360D2E775
:102160000020BDE8F08700BFA42D002010B5054C6D
:102170002046FFF76DF84FF0A0436365024BA3655F
:1021800010BD00BFA42D0020143600080378012BD9
:1021900070B5054650D12A4B446D98421BD1294B4E
:1021A0005A6B42F080025A635A6D42F080025A65BF
:1021B0005A6D5A6942F080025A615A6922F08002CF
:1021C0005A610E2143205B6900F0D6FB1E4BE36091
:1021D0001E4BC4F800380023C4F8003EC02323601F
:1021E0006E6D4FF40413A3633369002BFCDA0123F3
:1021F00033610C2000F040FE3369DB07FCD4122071
:1022000000F03AFE3369002BFCDA0026A66028466F
:10221000FFF740FF6B68C4F81068DB68C4F8146807
:10222000C4F81C684BB90A4BA3614FF0FF336361DC
:10223000A36843F00103A36070BD064BF4E700BF41
:10224000A42D00200038024040140040030020026A
:10225000003C30C0083C30C0F8B5446D0546002154
:102260002046FFF735FFA96D00234FF001128F685C
:10227000C4F834384FF00066C4F81C284FF0FF3023
:1022800004EB431201339F42C2F80069C2F8006BAD
:10229000C2F80809C2F8080BF2D20B686A6DEB6548
:1022A000636210231361166916F01006FBD1122029
:1022B00000F0E2FDD4F8003823F4FE63C4F80038DF
:1022C000A36943F4402343F01003A3610923C4F836
:1022D0001038C4F814380A4BEB604FF0C043C4F810
:1022E000103B084BC4F8003BC4F81069C4F800392F
:1022F000EB6D03F1100243F48013EA65A362F8BDAD
:10230000F035000840800010426D90F84E10D2F871
:10231000003823F4FE6343EA0113C2F80038704723
:102320002DE9F0410EB200EB86080D46D8F80C10EE
:102330000F6807F00303022B50D0032B50D03D4A07
:102340003D4F012B18BF1746446D4FEA451E04EB65
:102350000E030022C3F8102B8A6905F1100C002A25
:1023600040D04A8A05F158035B013A43E250012309
:10237000D4F81C2803FA0CF31343A6444A69C4F8A2
:102380001C380023CEF8103905F13F03002A39D05C
:102390000A8A898B9208012988BF4A43C16D04EBE0
:1023A0008303561841EA0242C66529465A60204610
:1023B000FFF78EFED8F80C301B8A43EA85531F4383
:1023C00005F148035B01E7500123D4F81C2803FA08
:1023D00005F51543C4F81C58BDE8F081174FB3E765
:1023E000174FB1E704EB4613D3F8002B22F4004259
:1023F000C3F8002BD4F81C28012303FA0CF322EABB
:102400000303BAE704EB83030E4A5A6004EB461653
:1024100029462046FFF75CFED6F8003923F4004336
:10242000C6F80039D4F81C38012202FA05F523EA6F
:102430000505CFE700800010008004100080081020
:1024400000800C1000040002826D1268C265FFF764
:1024500021BE00005831436D49015B5813F4004020
:1024600004D013F4001F14BF0120022070470000A5
:102470004831436D49015B5813F4004004D013F414
:10248000001F14BF012002207047000000EB8101F3
:10249000CB68196A0B6813604B6853607047000083
:1024A00000EB810330B5DD68AA691368D36019B900
:1024B000402B84BF402313606B8A1468426D1C4418
:1024C000013CB4FBF3F46343033323F0030302EB57
:1024D000411043EAC44343F0C043C0F8103B2B68AB
:1024E00003F00303012B09B20ED1D2F8083802EB36
:1024F000411013F4807FD0F8003B14BF43F08053A9
:1025000043F00053C0F8003B02EB4112D2F8003B0D
:1025100043F00443C2F8003B30BD00002DE9F04118
:10252000244D6E6D06EB40130446D3F8087BC3F8C8
:10253000087B38070AD5D6F81438190706D505EBF5
:1025400084032146DB6828465B689847FA072FD545
:10255000D6F81438DB072BD505EB8403D968CCB942
:102560008B69488A5E68B6FBF0F200FB12628AB99A
:102570001868DA6890420DD2121A83E814002023FA
:1025800083F311880B482146FFF78AFF84F31188F3
:10259000BDE8F081012303FA04F26B8923EA020308
:1025A0006B81CB6823B121460248BDE8F041184752
:1025B000BDE8F081A42D002000EB810370B5DD683B
:1025C000436D6C692668E6604A0156BB1A444FF4B5
:1025D0000020C2F810092A6802F00302012A0AB298
:1025E0000ED1D3F8080803EB421410F4807FD4F81E
:1025F000000914BF40F0805040F00050C4F80009BA
:1026000003EB4212D2F8000940F00440C2F800097E
:10261000D3F83408012202FA01F10143C3F8341857
:1026200070BD19B9402E84BF4020206020682E8ADA
:10263000841940F00050013C1A44B4FBF6F440EA1F
:10264000C440C6E7F8B504461E48456D05EB441383
:10265000D3F80869C3F80869F10717D5D5F8103819
:10266000DA0713D500EB8403D9684B691F68DA6871
:10267000974218D2D21B00271A605F60202383F391
:1026800011882146FFF798FF87F31188330617D585
:10269000D5F834280123A340134211D02046BDE8C9
:1026A000F840FFF71FBD012303FA04F2038923EA70
:1026B000020303818B68002BE8D021469847E5E7A9
:1026C000F8BD00BFA42D002096482DE9F84F456DB8
:1026D0006E69AB691E4016F4805F6E61044605D0DA
:1026E000FEF722FEBDE8F84F00F05ABC002E12DAC9
:1026F000D5F8003E8B489B071EBFD5F8003E23F05F
:102700000303C5F8003ED5F8043823F00103C5F8EB
:102710000438FEF733FE370502D58248FEF722FE65
:10272000B0040CD5D5F8083813F0060FEB6823F485
:1027300070530CBF43F4105343F4A053EB603107C4
:1027400004D56368DB680BB176489847F2025AD427
:10275000B3020CD5D4F85480DFF8C8A100274FF09D
:102760000109A36D9B68F9B28B4280F08780F70660
:1027700019D5616D0A6AC2F30A1702F00F0302F459
:10278000F012B2F5802F00F0A180B2F5402F0AD1EF
:1027900004EB830301F58051DB68186A00231A46B5
:1027A0009F4240F087803003D5F8184813D5E103E5
:1027B00002D50020FFF7B2FEA20302D50120FFF7E9
:1027C000ADFE630302D50220FFF7A8FE270302D562
:1027D0000320FFF7A3FE750384D5E00702D5002090
:1027E000FFF730FFA10702D50120FFF72BFF62079B
:1027F00002D50220FFF726FF23077FF573AF0320E2
:10280000FFF720FF6EE7D4F85480DFF818A1002707
:102810004FF00109A36D9B685FFA87FB5B4597D377
:1028200008EB4B13D3F8002902F44022B2F5802FB5
:1028300022D1D3F80029002A1EDAD3F8002942F069
:102840009042C3F80029D3F80029002AFBDB59463F
:10285000606DFFF73DFC228909FA0BF322EA0303BE
:10286000238104EB8B03DB689B6813B15946504608
:1028700098475846FFF736FC0137CBE708EB411283
:10288000D2F8003B03F44023B3F5802F10D1D2F8E7
:10289000003B002B0CDA628909FA01F322EA0303F8
:1028A000638104EB8103DB68DB680BB1504698471A
:1028B000013756E79C0708BF0A68072B98BF0270CC
:1028C00003F101039CBF120A013069E7023304EBF4
:1028D000830201F58051526890690268D0F808C0FF
:1028E0004068A2EB000E0022104697420AD104EB8A
:1028F000830463689B699A683A449A605A681744EB
:102900005F6050E712F0030F08BF0868964588BF64
:102910008CF8000002F1010284BF000A0CF1010CE6
:10292000E3E700BFA42D0020436D03EB4111D1F874
:10293000003B43F40013C1F8003B7047436D03EBC9
:102940004111D1F8003943F40013C1F80039704740
:10295000436D03EB4111D1F8003B23F40013C1F8A0
:10296000003B7047436D03EB4111D1F8003923F46C
:102970000013C1F80039704700F1604300F01F02F6
:10298000400903F5614309018000C9B200F16040CC
:1029900083F8001300F5614001239340C0F88031B3
:1029A0000360704730B5039C0172043304FB0325B8
:1029B000C361049B03630021059B00604060C1600C
:1029C000426102618561046242628162C162436365
:1029D00030BD00000022416A41610161C260826233
:1029E000C2626FF00101FEF7E9BF000003694269AE
:1029F000934203D1C2680AB100207047181D704786
:102A000003691960C2680132C260C26913448269F5
:102A10000361934224BF436A03610021FEF7C2BFF2
:102A200038B504460D46E3683BB16269131D126870
:102A3000A3621344E362002038BD237A33B92946E8
:102A40002046FEF79FFF0028EDDA38BD6FF0010049
:102A5000FBE70000C368C269013BC36043691344DC
:102A600082694361934224BF436A436100238362C6
:102A7000036B03B11847704770B52023044683F3F6
:102A80001188866A3EB9FFF7CBFF054618B186F379
:102A90001188284670BDA36AE26A13F8015BA3623D
:102AA000934202D32046FFF7D5FF002383F311881A
:102AB000EFE700002DE9F84F04460E469046994690
:102AC000202787F311880025AA46D4F828B0BBF147
:102AD000000F09D149462046FFF7A2FF20B18BF332
:102AE00011882846BDE8F88FA16AE36AA8EB050BB8
:102AF0005B1A9B4528BF9B46BBF1400F1BD9334651
:102B000001F1400251F8040B43F8040B9142F9D152
:102B1000A36A40334036A3624035A26AE36A9A4210
:102B200002D32046FFF796FF8AF311884545D8D295
:102B300087F31188C9E730465A46FEF71BF9A36AA6
:102B40005B445E44A3625D44E7E7000010B5029C6D
:102B50000172043303FB0421C36100238362C36257
:102B6000039B0363049B00604060C4604261026198
:102B7000816104624262436310BD0000026AC26068
:102B8000426A4261026100228262C2626FF0010108
:102B9000FEF714BF436902699A4203D1C2680AB1C1
:102BA00000207047184650F8043B0B607047000047
:102BB000C368C2690133C3604369134482694361D6
:102BC000934224BF436A43610021FEF7EBBE00003D
:102BD00038B504460D46E3683BB123691A1DA2626D
:102BE000E2691344E362002038BD237A33B92946F1
:102BF0002046FEF7C7FE0028EDDA38BD6FF0010071
:102C0000FBE7000003691960C268013AC260C2694B
:102C1000134482690361934224BF436A0361002322
:102C20008362036B03B118477047000070B520231F
:102C300004460E4683F31188856A35B91146FFF7BD
:102C4000C7FF10B185F3118870BDA36A1E70A36A17
:102C5000E26A01339342A36204D3E1692046043956
:102C6000FFF7D0FF002080F3118870BD2DE9F84FE9
:102C700004460D4691469A464FF0200888F3118885
:102C80000026B346A76A4FB951462046FFF7A0FF7A
:102C900020B187F311883046BDE8F88FA06AE76A53
:102CA000A9EB06033F1A9F4228BF1F46402F1BD99E
:102CB00005F1400355F8042B40F8042B9D42F9D14F
:102CC000A36A4033A3624036A26AE36A9A4204D3FD
:102CD000E16920460439FFF795FF8BF311884E45D3
:102CE000D9D288F31188CDE729463A46FEF742F853
:102CF000A36A3B443D44A3623E44E5E7026943695D
:102D00009A4203D1C3681BB9184670470023FBE7FA
:102D1000836A002BF8D0043B9B1AF5D01360C3687C
:102D2000013BC360C3691A44836902619A4224BFAC
:102D3000436A0361002383620123E5E700F072B96F
:102D4000034B002258631A610222DA60704700BF09
:102D5000000C0040014B0022DA607047000C00407C
:102D6000014B5863704700BF000C0040FEE70000B5
:102D700010B5174CFEF70CFDFEF72EFE802215490C
:102D80002046FEF7B3FD012344F8180C0374124BE0
:102D9000124AD96821F4E0610904090C0A43104978
:102DA000DA60CA6842F08072CA600E490A6842F06E
:102DB00001020A601022DA77202283F82220002301
:102DC00083F3118862B60848BDE81040FEF7B0BD35
:102DD000302600202036000800ED00E00003FA0550
:102DE000F0ED00E0001000E0283600082DE9F84F73
:102DF0001F4CDFF88090656904F114074FF000085C
:102E0000D9F82430266AAA689E1B96421DD34FF03B
:102E1000200AAA68236AD5F80CB0134423622B68F1
:102E2000BB425F60A6EB02066361C5F80C8001D16E
:102E3000FFF790FF88F311882869D8478AF3118833
:102E40006569AB689E42E4D2DAE76269BA420CD0A7
:102E5000916823628E1B9660A86802282CBF181800
:102E6000981CBDE8F84FFFF77BBFBDE8F88F00BFA7
:102E700008260020000C0040034B59685A68521A7B
:102E80009042FBD8704700BF001000E04B684360E1
:102E90008B688360CB68C3600B6943614B690362D5
:102EA0008B6943620B6803607047000008B5224BD2
:102EB00022481A6940F2FF110A431A611A6922F482
:102EC000FF7222F001021A611A691A6B0A431A632F
:102ED0001A6D0A431A651A4A1B6D1146FFF7D6FF91
:102EE000184802F11C01FFF7D1FF174802F1380121
:102EF000FFF7CCFF154802F15401FFF7C7FF144854
:102F000002F17001FFF7C2FF124802F18C01FFF7D6
:102F1000BDFF114802F1A801FFF7B8FF0F4802F109
:102F2000C401FFF7B3FF0E4802F1E001FFF7AEFF67
:102F3000BDE8084000F0E2B800380240000002405E
:102F4000483600080004024000080240000C02401D
:102F5000001002400014024000180240001C024011
:102F60000020024008B500F039FAFFF701FFFFF733
:102F700061F8BDE80840FEF739BE00007047000068
:102F8000064A536823F001035360EFF30983683363
:102F900083F30988002383F31188704730EF00E042
:102FA00010B5202383F31188104B5B6813F4006382
:102FB00018D0F1EE103AEFF309844FF0807344F823
:102FC0004C3C0B4BDB6844F8083CA4F1680383F3EA
:102FD0000988FEF76BFC18B1064B44F8503C10BD55
:102FE000054BFAE783F3118810BD00BF00ED00E048
:102FF00030EF00E03103000834030008084B1A6981
:10300000920710B508D500241C61202383F3118892
:10301000FFF7ECFE84F31188BDE81040FFF7C0BF56
:10302000000C0040104B1A6C42F008021A641A6E31
:1030300042F008021A660D4A1B6E936843F00803BB
:1030400093600B4B53229A624FF0FF32DA620022F8
:103050009A615A63DA605A6001225A6108211A6043
:103060003220FFF789BC00BF00380240002004E096
:10307000000C00401F4B1A696FEAC2526FEAD2522D
:103080001A611A69C2F308021A614FF0FF301A6917
:103090005A69586100215A6959615A691A6A62F07D
:1030A00080521A621A6A02F080521A621A6A5A6AC6
:1030B00058625A6A59625A6A1A6C42F080521A640B
:1030C0001A6E42F080521A661A6E0B4A106840F46B
:1030D00080701060186F00F44070B0F5007F1EBF64
:1030E0004FF4803018671967536823F400735360F6
:1030F00000F054B90038024000700040304B4FF0EF
:1031000080521A642F4A4FF4404111601A6842F00D
:1031100001021A601A689207FCD59A6822F003022D
:103120009A60274B19469A6812F00C02FBD1186876
:1031300000F0F90018609A601A6842F480321A6050
:103140000B689B03FCD54B6F43F001034B671C4B93
:103150005A6F9007FCD51C4A5A601A6842F0807278
:103160001A60184A53685904FCD5154B1A68920125
:10317000FCD5164A9A60164B1A68164B9A42164BA3
:103180001BD1164A1168164A914216D140F2051217
:103190001A600B4B9A6842F002029A609A6802F039
:1031A0000C02082AFAD15A6C42F480425A645A6ED0
:1031B00042F480425A665B6E704740F20572E7E760
:1031C00000380240007000400854400700948838DE
:1031D000002004E011640020003C024000ED00E00B
:1031E00041C20F41084A08B5536911680B4003F00A
:1031F0000103536123B1054A13680BB15068984726
:10320000BDE80840FFF7CCBE003C01408825002007
:10321000084A08B5536911680B4003F00203536173
:1032200023B1054A93680BB1D0689847BDE80840C0
:10323000FFF7B6BE003C014088250020084A08B5CB
:10324000536911680B4003F00403536123B1054A2D
:1032500013690BB150699847BDE80840FFF7A0BE5D
:10326000003C014088250020084A08B553691168D0
:103270000B4003F00803536123B1054A93690BB176
:10328000D0699847BDE80840FFF78ABE003C01407E
:1032900088250020084A08B5536911680B4003F0DF
:1032A0001003536123B1054A136A0BB1506A984762
:1032B000BDE80840FFF774BE003C014088250020AF
:1032C000174B10B55C691A68144004F478725A619F
:1032D000A30604D5134A936A0BB1D06A98476006D7
:1032E00004D5104A136B0BB1506B9847210604D5D7
:1032F0000C4A936B0BB1D06B9847E20504D5094A91
:10330000136C0BB1506C9847A30504D5054A936C18
:103310000BB1D06C9847BDE81040FFF741BE00BF2D
:10332000003C0140882500201A4B10B55C691A68E2
:10333000144004F47C425A61620504D5164A136DA8
:103340000BB1506D9847230504D5134A936D0BB10B
:10335000D06D9847E00404D50F4A136E0BB1506E40
:103360009847A10404D50C4A936E0BB1D06E9847D0
:10337000620404D5084A136F0BB1506F98472304B9
:1033800004D5054A936F0BB1D06F9847BDE8104044
:10339000FFF706BE003C014088250020062108B545
:1033A0000846FFF7E9FA06210720FFF7E5FA0621AC
:1033B0000820FFF7E1FA06210920FFF7DDFA0621D0
:1033C0000A20FFF7D9FA06211720FFF7D5FA0621C0
:1033D0002820BDE80840FFF7CFBA000008B5FFF786
:1033E00049FEFDF783FDFDF731FFFDF705FEFFF711
:1033F000C5FDBDE80840FFF7A1BC0000034611F879
:10340000012B03F8012B002AF9D170471210121377
:103410001211000053544D3332463F3F3F0000002D
:1034200000000000143400083F00000013040000F6
:10343000503400083F000000190400005A3400080E
:103440003F00000021040000643400083F00000039
:1034500053544D3332463430780053544D33324652
:103460003432780053544D33324634343658580091
:1034700000000000710F00085D0F0008990F0008A0
:10348000850F0008910F00087D0F0008690F0008E4
:10349000550F0008F50F00080000000001000000B3
:1034A0000000000002000000000000009D11000864
:1034B0000512000840004000E02A0020F02A002009
:1034C00002000000000000000300000000000000F7
:1034D000491200080000000010000000002B00202E
:1034E000000000000100000000000000A42D0020EA
:1034F000010102004C61736572204E61766967615B
:1035000074696F6E0025424F415244252D424C0094
:103510002553455249414C25000000008D1B0008F1
:10352000F51A000809110008711B0008430000008B
:103530003435000809024300020100C032090400CA
:103540000001020201000524001001052401000110
:10355000042402020524060001070582030800FF77
:1035600009040100020A00000007050102400000F2
:1035700007058102400000001200000080350008AD
:103580001201100102000040AC275211000201029A
:10359000030100000403090425424F415244250061
:1035A0005652427261696E2D7635320030313233B7
:1035B000343536373839414243444546000000002F
:1035C00000400000004000000040000000400000FB
:1035D00000000100000002000000020000000200E4
:1035E00000000200000002000000020000000200D3
:1035F0000000000091130008711600081D17000854
:1036000040004000042E0020042E00200100000095
:10361000142E002080000000400100000300000084
:103620006D61696E0000000040360008202E002009
:1036300018300020010000006D2D0008000000007F
:1036400069646C65000000000000802A0000000032
:10365000AAAAAAAA00000000FFFF000000000000C4
:1036600000A00A000000000000000000AAAAAAAA08
:1036700000000000FFFF000000000000000000004C
:103680000004000000000000AAAAAAAA000000008E
:10369000FFFF00000000000000000000000000101C
:1036A00000000000AAAAAAAA00000000FFFF000074
:1036B000000000000000000000000000000000000A
:1036C000AAAAAAAA00000000FFFF00000000000054
:1036D000000000000000000000000000AAAAAAAA42
:1036E00000000000FFFF00000000000000000000DC
:1036F0000000000000000000AAAAAAAA0000000022
:10370000FFFF0000000000000000000000000000BB
:10371000000000000A00000000000000030000009C
:103720000000000000000000000000000000000099
:103730000000000000000000000000000000000089
:103740000000000000000000FF00960000000008DC
:103750000400000094350008000000000000000094
:103760000000000000000000000000000000000059
:00000001FF
